:020000040000FA
:04000000CC303A289E
:040004000034003490
:08000800A000030EA100831209
:1000100005191128831601178312B2308100B1012E
:100020002C2883160113831203140B190310A80D37
:10003000A90DAA0DAB0DAC0DAC16FF302C02031DA3
:100040002C28FA302B02031D2C2832152A08AF0069
:100050002908AE002808AD008B100B11210E83007B
:06006000A00E200E0900B5
:0C007400203084008001840A80300402E7
:10008000031C3C289C2183160C30850587018312B4
:10009000850187010730990000309A0010308316DF
:1000A0008E008312603083168F0083120030831617
:1000B000910000008312C830831681008312313012
:1000C0009000003083168C00831210308B003E228B
:1000D00081018E018F010B118B100B108C018B177E
:1000E0007F2032198B20B40B7D280310851903144F
:1000F000BA0DF0303A0203191021952270286400DD
:100100003310B10A311F8A28AC01AB01AA01A90141
:10011000A801B101080032110130B7008B13203063
:10012000370783169B001C141A088312A400103092
:10013000370783169B001C141A088312A300A6001D
:100140000230A6060030370783169B001C141A08DD
:100150008312A200A7000130A7068B17331CB62814
:1001600022090339A200A309A409A50924082F0222
:10017000031D0A2923082E02031D0A2922082D0225
:10018000031D0A2901303702031DCB283E18CB2856
:100190003E143F14B72102303702031DD428BE1885
:1001A000D428BE143F14C32103303702031DDD28B9
:1001B0003E19DD283E153F14CF2104303702031DC0
:1001C000E628BE19E628BE153F14DB2105303702AC
:1001D000031DEF283E1AEF283E163F14E721063094
:1001E0003702031DF828BE1AF828BE163F14F22164
:1001F00007303702031D01293E1B01293E173F141A
:10020000FD2108303702031D0A29BE1B0A29BE172B
:100210003F140822B70A09303702031808008E2855
:100220000130B600B400B500B70085018701B213F4
:100230003B227F20B40B2929031085190314BA0D22
:10024000F0303A0203195129B50B29299630B5002F
:100250005D21321D19293211331C33292D0903392F
:10026000AD00AE09AF092F1C19292D083002031962
:1002700019292D08B0002E1E19298B13203037079D
:10028000BC002F08BB00872110303707BC002E08A8
:10029000BB00872100303707BC002D08BB00872139
:1002A0008B1785018701B70AB6010130B500093007
:1002B0003702031C19293E220800013037020319B6
:1002C00013220230370203191822033037020319B0
:1002D0001D22043037020319222205303702031988
:1002E00027220630370203192C2207303702031960
:1002F0003122083037020319362208003F1C08005B
:100300003F101030BC003E08BB00872108008B1353
:100310003B0883161C159A0083123C0883169B0029
:1003200055309D00AA309D009C1464009C189529AE
:100330001C1183128B170800831610309B001C14AD
:100340001A088312BE00831630309B001C141A0852
:100350008312DE00FF30C800CA15CB15CC15CD15B1
:10036000CE15CF15D015D115D215D3150800F13003
:10037000BE05FF30DE051130C405C0000030C200EC
:10038000C6005F100800F230BE05FF30DE05023007
:10039000C405C0000030C200C6005F100800F43081
:1003A000BE05FF30DE050630C405C0000030C200C7
:1003B000C6005F100800F830BE05FF30DE051830BB
:1003C000C405C0000030C200C6005F1008001F3026
:1003D000BE05C030DE058830C505C1000030C30051
:1003E000C70008002F30BE05C030DE051030C5053F
:1003F000C1000030C300C70008004F30BE05C03048
:10040000DE053030C505C1000030C300C70008005C
:100410008F30BE05C030DE05C030C505C1000030DC
:10042000C300C700080010308506023087060800A8
:100430002030850600308706080021308506003010
:100440008706080002308506023087060800003063
:1004500085060C30870608000030850601308706C7
:100460000800003085062130870608000030850628
:100470001830870608003E18132208003E18B721DE
:10048000BE18C3213E19CF21BE19DB213E1AE72138
:10049000BE1AF2213E1BFD21BE1B08220800B60138
:1004A000B401B5013D1C572ABD01BD14592ABD0137
:1004B0003D143D08B60064005D2A5E2A5F2A602A6A
:1004C000612AFF30B51B8500B51F8501B40B5B2A7F
:1004D000B50B5B2A0310B60CB608031D5B2A00306F
:1004E000BC003D08BB008721080005125C180516FA
:1004F000DC1C8512DC1885165C1D05105C190514C2
:10050000DC1D8510DC1985145C1E87105C1A8714AD
:10051000DC1E0711DC1A07155C1F07105C1B071493
:10052000DC1F8712DC1B871608008F0803190800E0
:100530008F0178308E00C80FBF2CC80A441CC52A12
:10054000461CB62ACA1CA72ACA014A15D32A4A1D24
:10055000AC2ACA01CA15D32ACA1DB12ACA014A1631
:10056000D32A4A1ED32ACA01CA14D32A4A1DBB2A37
:10057000CA014A16D32ACA1DC02ACA014A16D32A5A
:100580004A1ED32ACA01CA14D32ACA1CCA2ACA01BB
:100590004A15D32A4A1DCF2ACA01CA15D32A4A1E90
:1005A000D32ACA014A15C41CFA2AC61CEB2ACB1C42
:1005B000DC2ACB014B15082B4B1DE12ACB01CB15B7
:1005C000082BCB1DE62ACB014B16082B4B1E082B04
:1005D000CB01CB14082B4B1DF02ACB014B16082B5B
:1005E000CB1DF52ACB014B16082B4B1E082BCB013C
:1005F000CB14082BCB1CFF2ACB014B15082B4B1D12
:10060000042BCB01CB15082B4B1E082BCB014B1514
:10061000441D2F2B461D202BCC1C112BCC014C151F
:100620003D2B4C1D162BCC01CC153D2BCC1D1B2B73
:10063000CC014C163D2B4C1E3D2BCC01CC143D2B3C
:100640004C1D252BCC014C163D2BCC1D2A2BCC014F
:100650004C163D2B4C1E3D2BCC01CC143D2BCC1C01
:10066000342BCC014C153D2B4C1D392BCC01CC151A
:100670003D2B4C1E3D2BCC014C15C41D652BC61DBE
:10068000562BCD1C472BCD014D155F13732B4D1DE4
:100690004C2BCD01CD15732BCD1D512BCD014D16FE
:1006A000732B4D1E732BCD01CD14732B4D1D5B2B66
:1006B000CD014D16732BCD1D602BCD014D16732B27
:1006C0004D1E732BCD01CD14732BCD1C6A2BCD0188
:1006D0004D15732B4D1D6F2BCD01CD15732B4D1E5D
:1006E000732BCD014D155F1B9C2B441E9C2B461E6E
:1006F0008D2BCE1C7E2BCE014E15AA2B4E1D832B8F
:10070000CE01CE15AA2BCE1D882BCE014E16AA2BBC
:100710004E1EAA2BCE01CE14AA2B4E1D922BCE011B
:100720004E16AA2BCE1D972BCE014E16AA2B4E1E6F
:10073000AA2BCE01CE14AA2BCE1CA12BCE014E1576
:10074000AA2B4E1DA62BCE01CE15AA2B4E1EAA2BD0
:10075000CE014E15C51DD12BC71DC22BCF1CB32BEF
:10076000CF014F15DF2B4F1DB82BCF01CF15DF2B3E
:10077000CF1DBD2BCF014F16DF2B4F1EDF2BCF011F
:10078000CF14DF2B4F1DC72BCF014F16DF2BCF1DF3
:10079000CC2BCF014F16DF2B4F1EDF2BCF01CF14F9
:1007A000DF2BCF1CD62BCF014F15DF2B4F1DDB2BA3
:1007B000CF01CF15DF2B4F1EDF2BCF014F15451E6D
:1007C000062C471EF72BD01CE82BD0015015142CFB
:1007D000501DED2BD001D015142CD01DF22BD001C3
:1007E0005016142C501E142CD001D014142C501D53
:1007F000FC2BD0015016142CD01D012CD00150160A
:10080000142C501E142CD001D014142CD01C0B2CE2
:10081000D0015015142C501D102CD001D015142CC3
:10082000501E142CD0015015C51E3B2CC71E2C2C5D
:10083000D11C1D2CD1015115492C511D222CD10147
:10084000D115492CD11D272CD1015116492C511EEF
:10085000492CD101D114492C511D312CD1015116F3
:10086000492CD11D362CD1015116492C511E492C31
:10087000D101D114492CD11C402CD1015115492C46
:10088000511D452CD101D115492C511E492CD101A6
:100890005115451F712C471F622CD21C532CD201BD
:1008A0005215DF137F2C521D582CD201D2157F2CEC
:1008B000D21D5D2CD20152167F2C521E7F2CD201EC
:1008C000D2147F2C521D672CD20152167F2CD21DC0
:1008D0006C2CD20152167F2C521E7F2CD201D214C6
:1008E0007F2CD21C762CD20152157F2C521D7B2CD2
:1008F000D201D2157F2C521E7F2CD2015215DF1B44
:10090000A82CC51FA82CC71F992CD31C8A2CD30137
:100910005315B62C531D8F2CD301D315B62CD31DD4
:10092000942CD3015316B62C531EB62CD301D314DA
:10093000B62C531D9E2CD3015316B62CD31DA32CBD
:10094000D3015316B62C531EB62CD301D314B62C98
:10095000D31CAD2CD3015315B62C531DB22CD3018F
:10096000D315B62C531EB62CD30153157E21400847
:10097000C4004108C5005F18DF145F1CDF10480881
:10098000C9000C304A05031D05120C304B05031D30
:1009900085120C304C05031D05100C304D05031D50
:1009A00085100C304E05031D87100C304F05031DBC
:1009B00007110C305005031D07100C305105031DA5
:1009C00087120C305205031D07120C305305031D0E
:1009D000871149080E020318192D12304A05031D0C
:1009E000051612304B05031D851612304C05031DEC
:1009F000051412304D05031D851412304E05031DDC
:100A0000871412304F05031D071512305005031DC2
:100A1000071412305105031D871612305205031DAD
:100A2000071612305305031D8715FF3048020319BE
:100A300008008F08031D08007F2049080E02031CD0
:100A4000192D18304A05031D051206304A05031DED
:100A5000051618304B05031D851206304B05031D86
:100A6000851618304C05031D051006304C05031D76
:100A7000051418304D05031D851006304D05031D66
:100A8000851418304E05031D871006304E05031DD2
:100A9000871418304F05031D071106304F05031D3D
:100AA000071518305005031D071006305005031DAB
:100AB000071418305105031D871206305105031D18
:100AC000871618305205031D071206305205031D04
:100AD000071618305305031D871106305305031DF3
:040AE000871508006E
:084000000400030007000100A9
:02400E00CC33B1
:10420000010078007A007C007E007B0079007F004E
:104210007D007A0078007E007C007D007F007900C0
:104220001100F200F600FA00FE00F200F600FA00BB
:10423000FE00F200F600FA00FE00F200F600FA00BE
:10424000FF00050005000500050009000900090040
:1042500009000D000D000D000D00110011001100EE
:104260000000FF00FF00FF00FF00FF00FF00FF0055
:10427000FF00FF00FF00FF00FF00FF00FF00FF0046
:10428000FF007B00FF00FF00FF00FF00FF00FF00BA
:10429000FF00FF00FF00FF00FF00FF00FF00FF0026
:1042A000FF00FE00FF00FF00FF00FF00FF00FF0017
:1042B000FF00FF00FF00FF00FF00FF00FF00FF0006
:1042C000FF001100FF00FF00FF00FF00FF00FF00E4
:1042D000FF00FF00FF00FF00FF00FF00FF00FF00E6
:1042E000FF00FF00FF00FF00FF00FF00FF00FF00D6
:1042F000FF00FF00FF00FF00FF00FF00FF00DD00E8
:00000001FF
